:100000000C9496010C94BE010C94BE010C94BE019C
:100010000C94BE010C94BE010C94BE010C94BE0164
:100020000C94BE010C9437030C941A230C94CC212D
:100030000C94BE010C94BE010C94BE010C94BE0144
:100040000C94540A0C94BE010C94BE010C94BE0195
:100050000C94BE010C94BE010C94BE010C94E819E2
:100060000C94BE010C94C11E0C94041F0C94BE0190
:100070000C94BE010C94BE010C94BE010C94BE0104
:100080000C94BE010C94BE010C94BE010C94BE01F4
:100090000C94BE010C94BE010C94BE010C94BE01E4
:1000A0000C94BE010C94BE010C94BE018B129112F3
:1000B00097129E12AC12CE12EC12F11AF41AE71A31
:1000C000EB1A151B151B151BF81AFC1A001B061B37
:1000D0000A1B151B101B434C49206E6F7420617660
:1000E00061696C61626C652C2075736520636F6E4D
:1000F000666967757261746F72210000000002000A
:10010000080E0000030401000B00000000000000C6
:100110000000000000000000000408020110408000
:1001200040102040804080080204018040201002DE
:10013000011080102040400404040404030405025C
:100140000202020403020202020606060606060472
:100150000402020204000000002300260029002CF3
:10016000002F0000000000250028002B002E003189
:100170000000000000240027002A002D00300008A5
:100180000B0002020201000904000001020200004B
:1001900005240010010524010101042402060524A0
:1001A0000600010705810310004009040100020A4E
:1001B000000000070502024000000705830240001E
:1001C0000000C18081C112010002020000404123F1
:1001D000368000010102000112010002000000400F
:1001E0004123368000010102000118034100720022
:1001F0006400750069006E006F0020004C004C0028
:1002000043002203410072006400750069006E0023
:100210006F0020004C0065006F006E0061007200EE
:1002200064006F00040309040000000000000000E7
:100230002A2B280000000000000000000000000041
:1002400000000000000000002C9EB4A0A1A2A43475
:10025000A6A7A5AE362D3738271E1F20212223241E
:100260002526B333B62EB7B89F8485868788898ABA
:100270008B8C8D8E8F909192939495969798999A56
:100280009B9C9D2F3130A3AD350405060708090A54
:100290000B0C0D0E0F101112131415161718191A36
:1002A0001B1C1DAFB1B0B500090402000103000022
:1002B00000092101010001226500070584034000B7
:1002C0000105010902A1010901A100850105091922
:1002D000012903150025019503750181029501751A
:1002E00005810305010930093109381581257F751C
:1002F0000895038106C0C005010906A10185020514
:100300000719E029E7150025017501950881029577
:1003100001750881039506750815002565050719FF
:100320000029658100C0A21CF21FB62411241FBE43
:10033000CFEFDAE0DEBFCDBF12E0A0E0B1E0E8E150
:10034000FCE402C005900D92AA35B107D9F715E07B
:10035000AAE5B2E001C01D92A831B107E1F713E0B0
:10036000CCE2D3E004C02297FE010E947F25C63272
:10037000D107C9F70E942E200C940A260C94000085
:1003800080910008909101088737974709F0A89558
:100390000895DC01ED91FC910190F081E02D09952B
:1003A000089520919C0330919D03382748E0C901AE
:1003B000880F991F37FF06C09C0151E2252750E1A5
:1003C000352701C09C01415091F730939D03209344
:1003D0009C03089588E380939E0380E092ECA1E063
:1003E000B0E080939F039093A003A093A103B093E8
:1003F000A20387E08093AB0380EC9AECA9E8B6E314
:100400008093A3039093A403A093A503B093A603A2
:1004100085E08093AC038DEE9EEFADEABEED809358
:10042000A7039093A803A093A903B093AA03EDEAAE
:10043000F3E080E090E0863028F4DC01AC5DBD4F55
:100440002C9101C020E0219301968831910599F704
:1004500082E08093C5038AE08093C603089580EC10
:1004600097EFAAEBB7E38093E3039093E403A093A1
:10047000E503B093E60380E090E0A0E0B0E5809370
:10048000E7039093E803A093E903B093EA03EBEE4C
:10049000F3E080E081938F5F8031E1F70895A0E081
:1004A000B0E0E5E5F2E00C944825D82F0E943E1A12
:1004B0006115710581059105C9F30E94EB25109224
:1004C000A7031092A8031092A9031092AA03C4E0F4
:1004D000812C912C54018A94C090A703D090A8033A
:1004E000E090A903F090AA03FE2CED2CDC2CCC2488
:1004F0000E94E625A50194010E9427256C0D7D1D13
:100500008E1D9F1D6093A7037093A8038093A9037A
:100510009093AA03C15001F7DD2309F450C00DEAFE
:1005200013E0E801A12CB12C62E3C62ED12CE12C02
:10053000F12C8881882309F442C0B39419F40E94F5
:10054000EA013DC00E94E625A70196010E942725E9
:10055000E1E0E60FADEAB3E08A2F801B8A1520F4B4
:100560008D918E13F9CFE9CF2091AC0330E0A0E15B
:10057000B7E20E94BF249B01AC01AE2FB0E00E9405
:10058000CE244090A3035090A4036090A5037090E4
:10059000A603640D751D861D971D4090E3035090C2
:1005A000E4036090E5037090E6034616570668067C
:1005B000790618F2E993A39488E1A812BACFCDB7CF
:1005C000DEB7E0E10C94642580919B03813019F43F
:1005D00082E080939B0380919B03833019F484E035
:1005E00080939B03089588E08093C10061E08AE0D6
:1005F0000E94161B60E08AE00E944F1B089500973E
:10060000C9F09C0140E050E068E478EE81E090E0C1
:100610000E9427252F3F31054105510529F020F083
:100620002FEF30E040E050E02093D1008091C000F7
:10063000806103C08091C0008F7E8093C0000895C8
:10064000219A229A239860E08BE00E94161B61E0B9
:100650008CE00E94161B0895EBE6F0E08081806834
:100660008083E8E6F0E080818160808308951F92B6
:100670000F920FB60F9211242F933F934F935F93D6
:100680006F937F938F939F93AF93BF93EF93FF935A
:100690001F9B0E94E402FF91EF91BF91AF919F9148
:1006A0008F917F916F915F914F913F912F910F901B
:1006B0000FBE0F901F901895A1E0B0E0E2E6F3E0C6
:1006C0000C9455251FB791E090939A03F894898371
:1006D0000E94C00198E1909360008981809360003E
:1006E00081110E94C0011FBF2196E3E00C94712587
:1006F0008F929F92AF92BF92CF92DF92EF92FF9232
:10070000CF93FC01C0A5EC2FE770F0E0E45EFD4F55
:10071000A081B0E0C7FF03C024E130E002C02FE0B9
:1007200030E0FC0197A183E1989FF0011124E25C85
:10073000FE4F80809180A280B380A20FB31F20E47F
:100740003FE14DE750E00E94D924A50194010E94A9
:1007500005258C2F887149F469017A01E0EDCE0EF0
:10076000E7E0DE1EE11CF11C1BC0C7FF05C060E412
:100770007AE88CE29EE004C060E07EEE8AEB9BE0CB
:1007800069017A01F8EBCF0EFBE0DF1EE11CF11CE2
:10079000A50194010E940525C20ED31EE41EF51E7C
:1007A000C701B60169517C4F8F4F9F4F28EE33E050
:1007B00040E050E00E940525A8EEB3E00E94CE2460
:1007C000CF91FF90EF90DF90CF90BF90AF909F9030
:1007D0008F9008958F3F910551F048F0811522E0E8
:1007E000920738F08115934030F482E0089580E05C
:1007F000089581E0089583E00895A0E0B0E0E3E08B
:10080000F4E00C945125EB018A01B82FB695A0E0D5
:1008100028813981F80120832A813B8121832C8121
:100820003D8122832E813F812383688179814A81A2
:100830005B812C813D81EE81FF819F2F9295990FE5
:10084000990F907C272F2370922B252F2370220F36
:10085000220F922B232F23702295207F922BF801B9
:1008600094830B5F1F4F2896AF5FBA1788F680FFFF
:1008700024C0888199810E94EA03D82E8A819B81B5
:100880000E94EA03E82E8C819D810E94EA03F82EE3
:100890008E819F810E94EA03F0E4DF9EA001112473
:1008A00090E1E99E90011124242B282BE4E0FE9E88
:1008B000B0011124262BF8012083CDB7DEB7E7E085
:1008C0000C946D25803223E0920708F1883E23E0E6
:1008D000920740F48F519340E4E096958795EA950E
:1008E000E1F70895803D27E0920718F48C5D93406E
:1008F0000895883928E0920768F4885C974074E08E
:10090000969587957A95E1F78D509C4F089580E0F4
:1009100090E008958FEF93E008958C30910540F4B6
:10092000A4E0880F991FAA95E1F7885D9C4F089570
:10093000843F23E0920718F484529C4F0895811558
:1009400024E0920740F48657934FF4E0880F991FF4
:10095000FA95E1F7089580E998E008959C013695AD
:10096000279525753575821B930B9C012373337373
:10097000969587959695879583739373820F931FAA
:100980009C0154E0369527955A95E1F7280F391FB9
:100990002F703F7041E051E0249FC001259F900DD2
:1009A000349F900D1124892F08952998882319F0D8
:1009B00000002A9A02C000002A980000299A00002C
:1009C0000895299A000083B12998000083FB8827A5
:1009D00080F90895CF93DF93D82F5E9A29985E9877
:1009E000C8E08D2F80780E94D504DD0FC150C9F773
:1009F0002998DF91CF9108958F770E94EA04089596
:100A0000CF93DF93D82FC8E08D2F80780E94D50434
:100A1000DD0FC150C9F72998DF91CF910895CF9389
:100A2000DF932998C8E080E0D82FDD0F0E94E10411
:100A30008D0FC150C9F7DF91CF9108950E94FC043A
:100A40000E940F055E9A0895A1E0B0E0EAE2F5E0A9
:100A50000C945625806869830E94EA046981862F78
:100A60000E9400055E9A2196E2E00C947225CF93D5
:100A7000C091A703C827E82FF0E0E256FC4F678536
:100A800089E70E9424056C2F8DE30E9424056C2FBA
:100A900082E40E942405CF91089586E20E941E05FB
:100AA0000895CF93DF93EC016C818CE10E942405C3
:100AB0006D818DE10E9424056E818EE10E942405E6
:100AC0006F8180E20E942405688581E20E942405EE
:100AD000698582E20E9424056A8583E20E942405DA
:100AE0006B8584E20E9424056C8585E20E942405C2
:100AF0006D858AE20E9424056E858EE60E9424059B
:100B00006F858FE60E942405688980E70E9424058E
:100B1000698981E70E9424056A8982E70E94240589
:100B2000DF91CF910895CF92DF92EF92FF92CF9312
:100B3000DF936B017C01C11488E3D8068CE9E806D9
:100B40008CE1F80628F5C701B60120E836E948E946
:100B500050E00E940525E901689760E879E687E69C
:100B60009FEF0E94E1246C0D7D1D8E1D9F1DF2E004
:100B7000660F771F881F991FFA95D1F721E732E09A
:100B800040E050E00E940525F22EE32E80E421C0D3
:100B9000C701B60120E03DE241E351E00E94052596
:100BA000E901689760E073ED8EEC9EEF0E94E1240E
:100BB0006C0D7D1D8E1D9F1D660F771F881F991F51
:100BC00021E732E040E050E00E940525F22EE32EBE
:100BD00080E66C2F6F71680F85E70E9424056E2DEB
:100BE00086E70E9424056F2D87E70E942405DF9188
:100BF000CF91FF90EF90DF90CF900895682F8DE612
:100C00000E94240508958F929F92AF92BF92CF9237
:100C1000DF92EF92FF92CF93DF93D82F83E00E9471
:100C20001E058093990384E00E941E05809398031B
:100C300060E086E00E94240561E087E00E942405D0
:100C40006FE789E00E94240565E08AE00E942405A0
:100C500065E18BE00E94240562E18CE00E9424059E
:100C60006DEF8DE00E94240560E08EE00E94240577
:100C7000DD2319F08BE291E008C02091C50333E138
:100C8000239FC0011124825C9E4F0E9451056CE895
:100C900080E30E9424056FE082E30E94240562E461
:100CA00083E30E9424058091C60387FF02C064E1AC
:100CB00001C06AE084E30E9424056AE285E30E94A1
:100CC00024056DE286E30E94240564ED87E30E941B
:100CD000240560E088E30E94240560E089E30E9427
:100CE0002405D11109C0C090A703D090A803E090BB
:100CF000A903F090AA0307C0C5E9CC2EC1ECDC2EF5
:100D0000ED2CCEEDFC2ECAE38F2C9924AA24BB2413
:100D1000682D8C2F0E942405682D85E08C0F0E9481
:100D20002405FE2CED2CDC2CCC24CF5FCE3361F7D8
:100D30006FEF83E40E9424056FEF84E40E94240592
:100D40006FEF85E40E9424056FEF86E40E9424057E
:100D5000DD2311F066E002C06091AB038DE60E94D6
:100D6000240560E089E70E9424056091AC038AE7CE
:100D70000E94240560E083E70E94240560E084E788
:100D80000E942405D11109C06091A3037091A403AE
:100D90008091A5039091A60304C060EC7AEC89E8E9
:100DA00096E30E949305DF91CF91FF90EF90DF9043
:100DB000CF90BF90AF909F908F90089561E087E0B3
:100DC0000E94240564E28EE70E94240563E088E027
:100DD0000E94240560E088E00E94240565E087E029
:100DE0000E94240562E085E00E94240583E00E94C1
:100DF0001E058093990384E00E941E05809398034A
:100E0000089583E00E941E058093990384E00E9468
:100E10001E058093980361E087E00E9424056AE044
:100E200070E080E090E00E94611A0E94DE060000FF
:100E30000895CF92DF92FF920F931F93CF93DF938A
:100E40001F92CDB7DEB7082F162F8EE399830E942D
:100E50002405F02EC02E9981D92E8C2D8F19811743
:100E600038F4F60161916F018FE70E942405F5CFF8
:100E700064E085E00E94240583E00E941E058093C3
:100E8000990384E00E941E05809398030E943E1AF5
:100E900060939403709395038093960390939703C4
:100EA00069E087E00E94240581E080939B030F9016
:100EB000DF91CF911F910F91FF90DF90CF90089518
:100EC0000F931F930E94190780919B03813099F41F
:100ED0000E943E1A0091940310919503209196036D
:100EE00030919703601B710B820B930B603A76482D
:100EF0008140910548F380919B03813031F467EA8A
:100F000071E086E094E00E94461D1F910F910895C4
:100F10000F931F9380919B03823021F410929B03C7
:100F200081E020C080919B038130D9F40E943E1A59
:100F300000919403109195032091960330919703AB
:100F4000601B710B820B930B613A764881409105CF
:100F500040F061E087E00E94240510929B0382E04C
:100F600001C080E01F910F910895CF93DF93EC01B2
:100F70004AE050E06D2F70E086E094E00E940B1E86
:100F80006EE286E094E00E94181DBE0184E0769532
:100F900067958A95E1F76F7077274AE050E086E021
:100FA00094E00E940B1E6EE286E094E00E94181D01
:100FB000BE016F7077274AE050E086E094E00E941F
:100FC0000B1EDF91CF910895D82FC0E0CD1780F48C
:100FD0005F9A64E670E080E090E00E94611A5F989A
:100FE00064E670E080E090E00E94611ACF5FEECF8F
:100FF0006CE271E080E090E00E94611AE6CF0F930E
:101000001F93CF93DF93EC01062F15E0115051F0A1
:10101000CE010E94F425081741F0602FCE010E94F6
:10102000FC25F4CF82E00E94E407DF91CF911F916D
:101030000F910895A0E0B0E0E0E2F8E00C944825BC
:10104000482E562EC0E0D0E0612C712CE12CF12C02
:1010500000E010E041100CC06090FC0386E4689E44
:101060003001112459E1E52EF12C02EE13E01EC0EF
:1010700091E049120FC06090FC03E6E46E9E3001DF
:101080001124FBE16F0E711C49E2E42EF12C0EE9F4
:1010900013E00CC082E0481209C028E1622E7724D8
:1010A0007394EE24E394F12C0BEF13E043018C0EC8
:1010B0009D1E10929D0310929C033401A62CA8182B
:1010C000B12CC30101966C01AE14BF04A8F4A00EAC
:1010D000B11E511006C0C3010E94F425F5018083A2
:1010E00005C0F5016081C3010E94FF07F501808101
:1010F0000E94D1013601E2CFC301511018C0C301D3
:101100000E94F425B82EC6010E94F4252B2D30E054
:10111000322F2227282B80919C0390919D038217C8
:10112000930779F4C0E0D0E05524539493CF36016F
:1011300060919D030E94FF0760919C03C6010E947D
:10114000FF07C05EDE4FC13E92E0D90708F482CFB0
:10115000852DCDB7DEB7E0E10C94642561E082E037
:101160000E941A08089560E082E00E941A088091A7
:10117000FB03853020F01092FB030E94AE088091A3
:10118000FB038093FC03089561E080E00E941A084D
:1011900061E081E00E941A08089560E080E00E940A
:1011A0001A08882351F060E081E00E941A08882321
:1011B00021F080919E03883349F00E942F020E9403
:1011C000EA0181E00E944F020E94C4080895CF9373
:1011D000C82F0E943E1A609358037093590380935E
:1011E0005A0390935B03C0936D03CC2329F040E036
:1011F00051EE60E070E004C040E855E260E070E06D
:1012000088E594E00E94711FCF91089590915C034E
:10121000492F4F7050E0BA016F5F7F4F292F30E0A8
:10122000E4E035952795EA95E1F76217730759F0E1
:10123000FA01E35AFC4F808381E0890F8F70907F21
:10124000892B80935C0308956EE770E088E594E055
:101250000E94C9010895A3E1B1E0E1E3F9E00C9433
:101260004925EDEAF3E0712C8191882321F07394F4
:1012700028E17212F9CF63EB71E086E094E00E94FE
:10128000461D4AE050E0672D86E094E00E94121E61
:1012900080E00E9403060E94DE068E010E5F1F4F53
:1012A000C12CD12C7601C39466246A945C2C0E94D4
:1012B000321A4B015C012091AC0330E0A0E1B7E2AF
:1012C0000E94BF249B01AC01C701B6010E94E1242A
:1012D0002091A3033091A4034091A5035091A6034C
:1012E000620F731F841F951F2091E3033091E40365
:1012F0004091E5035091E603261737074807590741
:1013000018F4F801608225C08C2D0E94370561E039
:1013100070E080E090E00E94611AF80110820E9463
:10132000321A681979098A099B09643F714081055D
:10133000910540F40E944D05F8019081981778F7C7
:101340008083EDCF50FE03C046985F9A02C0469A54
:101350005F982FEFC21AD20AE20AF20A0F5F1F4FFC
:101360008FEFC816D104E104F10409F09FCFCE013C
:101370009395FC01D82E7FEF68EC2E2F281B2715A4
:1013800010F051E056C0DE01129651E02FEF41E01F
:101390003D91321710F0322F01C0452F5F5F5F3F44
:1013A00011F0232FF5CF4193242F30E0A1E0B0E0DE
:1013B000AC0FBD1FA20FB31F5C93413079F0DE016B
:1013C000A20FB31F5C93423049F0AFEFBFEFAC0FF9
:1013D000BD1FA20FB31F6C934E3F78F6A2E0B0E0A2
:1013E000AC0FBD1FA20FB31F7C934D3F30F6A3E09F
:1013F000B0E0AC0FBD1FA20FB31F6C93BECF452F43
:10140000242F30E0FC01E20FF31F6081AFEFB0E06A
:10141000AC0FBD1FA20FB31F2C91621748F44150AF
:10142000DC01A40FB11D2C9120836C934111E8CFF6
:101430005F5F571520F3372D369520E0231770F4A2
:10144000DC01A20FB11D4C91522F530FFC01E50F8F
:10145000F11D50815C9340832E5FF0CFFDEAEF2EAB
:10146000F3E0FF2E8C01802F8D19871598F4F80179
:10147000C1908F014AE050E06C2D86E094E00E941C
:10148000031E6CE286E094E00E94181DF701C192F1
:101490007F01E9CF86E094E00E94201D81E0CD5ECF
:1014A000DE4FEFE00C9465251F920F920FB60F925E
:1014B00011241F932F933F934F935F936F937F93C9
:1014C0008F939F93AF93BF93CF93DF93EF93FF934C
:1014D000C0918600D09187008091170390911803E6
:1014E00020913903211155C09E01281B390B809191
:1014F000E7039091E803A091E903B091EA0385FD29
:1015000002C036952795253C49E03407B8F1409153
:101510000A0150E060E070E02CE1B695A795979540
:1015200087952A95D1F70097A105B10521F481E0AF
:1015300090E0A0E0B0E084179507A607B707D8F4BD
:1015400080910A018F3FB9F040E080910A0148176D
:1015500080F4842F90E0880F991FFC01E75EFC4F18
:1015600020813181FC01E55FFE4F318320834F5F95
:10157000ECCF10923A0310920A010BC02D3B82E08F
:10158000380720F080910A018031D8F08FEF8093E6
:101590000A01D0931803C0931703FF91EF91DF91D5
:1015A000CF91BF91AF919F918F917F916F915F91FB
:1015B0004F913F912F911F910F900FBE0F901F9051
:1015C000189510910A0181E0810F80930A01C901E9
:1015D0000E946204E12FF0E0EE0FFF1FE75EFC4F78
:1015E00091838083D6CF83E0809380008AE98093C3
:1015F00081008091E70386FD05C0809181008064B1
:10160000809381008FEF9FEF9093890080938800F3
:1016100080916F00806280936F0008950E94B308EC
:101620008091FC03843011F41092FC0308956F3014
:1016300018F086958058089589E0689F802D1124C0
:101640000895A0E0B0E0E7E2FBE00C945025C82F3D
:101650000E943E1A0091C8021091C9022091CA024C
:101660003091CB026B017C01C01AD10AE20AF30A65
:101670009701860149E8C41643E1D406E104F10468
:1016800010F01092CC026093C8027093C90280934C
:10169000CA029093CB02209139038FEF820F8230E0
:1016A000D8F5E091CC02EE2309F44EC1E13011F4FB
:1016B00082E0B8C1E03108F034C181E08E0F809340
:1016C000CC02F0E0E75EFC4FC083803109F0ACC192
:1016D000EBE1F3E0213029F4A181A695A695808164
:1016E00008C080819181A92FA695A695A69596956B
:1016F0008795A03148F4B0E090E0AA0FBB1FA55F2A
:10170000BE4F11969C938E9310923A03329683E0CB
:10171000E932F807F9F688C1233009F005C1E091F4
:10172000CC02E11104C0CF3009F07EC10DC1E83117
:1017300048F481E08E0F8093CC02F0E0E85EFC4F2D
:10174000C08372C1E83109F0ECC0C111EAC040E0C9
:1017500050E0ABE0CA01B3E0880F991FBA95E1F7FA
:10176000A49F9001A59F300D1124F901E75EFC4F65
:101770006081E1817E2F777075956795FC01EE0F92
:10178000FF1FE55FFE4F71836083F901E65EFC4F4A
:10179000B081B695B695B695E181FE2FF295FF0F13
:1017A000F07E6F2F6B2BE695E695E6957E2F777092
:1017B00075956795FC01EE0FFF1FE35FFE4F718388
:1017C0006083F901E55EFC4FB081B295B695B695A0
:1017D000B370C181DC2FDD0FDD0F6D2F6B2BC29538
:1017E000C695C695C370E281E170EE0FEE0F7E2FB5
:1017F0007C2B75956795FC01EE0FFF1FE15FFE4F97
:1018000071836083F901E35EFC4FB081B695E1819D
:10181000FE2FF795FF27F7956F2F6B2BE6957E2F01
:10182000777075956795FC01EE0FFF1FEF5EFE4F19
:1018300071836083F901E25EFC4FB081B295BF70A5
:10184000E181FE2FF295F07F6F2F6B2BE295EF7009
:101850007E2F777075956795FC01EE0FFF1FED5E8B
:10186000FE4F71836083F901E15EFC4FB081BB1FC5
:10187000BB27BB1FC181DC2FDD0F6D2F6B2BCC1F56
:10188000CC27CC1FE281E370EE0F7E2F7C2B759569
:101890006795FC01EE0FFF1FEB5EFE4F71836083C7
:1018A000F901EF5DFC4FB081B695B695E181FE2F51
:1018B000F295FF0FFF0FF07C6F2F6B2BE695E695EF
:1018C0007E2F777075956795FC01EE0FFF1FE95E1F
:1018D000FE4F71836083F901EE5DFC4F20812295FC
:1018E000269527703181E32FEE0FEE0FEE0F6E2F4E
:1018F000622B732F72957695777075956795FC01BD
:10190000EE0FFF1FE75EFE4F718360834F5F5F4FF7
:101910004230510509F01ECF80912F0383FF1092B2
:101920003A031092CC0280C0243009F07DC060914F
:10193000CC0261110BC0C83AB1F410929D03109211
:101940009C0388EA0E94D10181E06CC0613019F4E7
:10195000C093C70204C0623031F4C093C6028C2F1A
:101960000E94D1015AC0E091C6022E2F30E0220F12
:10197000331F462F50E0C9010296841795073CF0AB
:10198000633268F7FA01EA5EFC4FC083E8CF2D5F4F
:101990003F4F8C2F90E060919C0370919D03421704
:1019A000530749F4982F88278627972790939D03FC
:1019B00080939C0332C06817790769F58091C7024C
:1019C000813049F5E13118F080E18093C602F09052
:1019D000C602CAE1D3E000E010E00F15D0F4FE012A
:1019E0003197808190E0982F88272881822B63E0AF
:1019F000969587956A95E1F70E946204F801EE0FCB
:101A0000FF1FE55FFE4F918380830F5F1F4F22967C
:101A1000E4CF10923A031092CC028091CC0288233A
:101A200019F08F5F8093CC02CDB7DEB7E8E00C945D
:101A30006C25E82FF0E0EE51FC4FE185E03150F4E9
:101A4000F894F0E0EE0FFF1FE55FFE4F808191817B
:101A500078940895E03121F0E13169F483E001C028
:101A600082E00E94821B892B19F084EF93E0089595
:101A70008CE090E0089580E092E00895A2E2B0E06A
:101A8000E4E4FDE00C9446259E012F5F3F4F80E18A
:101A9000D9011D928A95E9F761EE71E086E094E044
:101AA00029A33AA30E94461D0E9401071D8A1E8A8F
:101AB0001F8A188E312C212C00E0812C912C54018E
:101AC00070EC472E7DE9572E78E5672E75E3772E6B
:101AD000E0E5CE2EE3ECDE2EE12CF12C84EF91E05C
:101AE000A0E0B0E08D8F9E8FAF8FB8A380EC97EF12
:101AF000AAEBB7E3898F9A8FAB8FBC8F80EC9DE9FF
:101B0000A8E5B5E3898B9A8BAB8BBC8B86E094E020
:101B10000E94AB1B892B09F4E1C086E094E00E948F
:101B2000CF1B9C0133272C32310509F442C0ACF4A1
:101B30002332310509F0ABC019821A821B821C8244
:101B40001D821E821F82188619861A861B861C8695
:101B50001D861E861F86188A60C02434310529F030
:101B60002335310509F4B2C092C064E486E094E004
:101B70000E94181D2AE030E040EC5DE968E575E35D
:101B800086E094E00E94A61D6CE286E094E00E944C
:101B9000181D2AE030E040EC57EF6AEB77E386E06F
:101BA00094E00E94A61D6CE286E094E00E94581D1D
:101BB000ADCF0F5F043009F0A9CF29813A814B8165
:101BC0005C81A8EEB3E00E94CE24698B7A8B8B8B6C
:101BD0009C8B2D813E814F8158850E94CE24698F38
:101BE0007A8F8B8F9C8F29853A854B855C852D8FCD
:101BF0003E8F4F8F58A32D853E854F8558890E9473
:101C0000CE246B017C0160323EE4730781059105AF
:101C100030F462E38CE10E94240500E077CF60336A
:101C200045E774078105910510F462E2F3CF603453
:101C30005CE975078105910510F466E2EBCF80E55C
:101C4000C81683ECD806E104F10410F462E1E2CF97
:101C500090E6C9169AEED906E104F10410F465E1A4
:101C6000D9CFA0E7CA16A1E1DA06A1E0EA06F1049D
:101C700010F461E0CFCFB0EACB16B6E8DB06B1E0F6
:101C8000EB06F10410F463E0C5CF65E0C3CF10EDBF
:101C9000180F1A3008F03ACFE1E0F0E0EC0FFD1F2A
:101CA00024E0029FE00DF11D112420813181428149
:101CB0005381AAE0B0E00E94CE24610F711D811D06
:101CC000911D608371838283938320CF49885A88D2
:101CD0006B887C88812C912C540118CF811491043D
:101CE000A104B10489F4C301B2010E94930561E02B
:101CF00070E080E090E00E94611A1D8A1E8A1F8AAF
:101D0000188E312C22242A948D8D9E8DAF8DB8A1F2
:101D100088169906AA06BB06D0F40E944D052D89A7
:101D20003E894F89588D280F311D411D511D2D8B26
:101D30003E8B4F8B588F381608F4382E821508F4D6
:101D4000282E3FEF831A930AA30AB30A56C0C30191
:101D5000B20128EE33E040E050E00E940525BA01D0
:101D6000A9012AE030E086E094E00E94F41D6CE2D4
:101D700086E094E00E94181D4AE050E0632D86E062
:101D800094E00E94031E6CE286E094E00E94181D1D
:101D90006D897E898F89988DA50194010E94052502
:101DA000BA01A9012AE030E086E094E00E94F41D27
:101DB0006CE286E094E00E94181D4AE050E0622D3B
:101DC00086E094E00E94031E6CE286E094E00E94AC
:101DD000581D4C0C5D1C6E1C7F1C898D9A8DAB8D23
:101DE000BC8D84159505A605B70520F449885A8849
:101DF0006B887C88812C912C540129893A894B89E4
:101E00005C89283E33404105510509F07FCEA296FA
:101E1000E2E10C946225ACE1B0E0E1E1FFE00C947A
:101E200050250E943E1A6B017C0181E00E9403064E
:101E300014E703E0198361E0CE0101960E94600778
:101E400000939B030E94DE066AEF70E080E090E062
:101E50000E94611A80919B03833089F486E094E0AC
:101E60000E94AB1B892B59F40E943E1A6C197D0904
:101E70008E099F096038734C894C9140D8F280914B
:101E80009B03833009F44FC08FE70E94FC040E943B
:101E90000F058983843511F083E05CC00E940F0533
:101EA00010926E0380936F030E940F0520916E03C2
:101EB00030916F03280F311D30936F0320936E0311
:101EC0000E940F05809370030E940F058093710399
:101ED000813110F7F12C0F2D10E08091710390E00B
:101EE000880F991F0817190740F40E940F05F80181
:101EF000EE58FC4F8083F394EECF80E7898361E056
:101F0000CE0101960E94600783E080939B030E94AC
:101F1000DE0662E370E080E090E00E94611A80914A
:101F20009B03833011F482E015C08FE70E94FC040C
:101F30000E940F058983803509F0AECF07EC13E0CE
:101F40000E940F05F80181938F01F3E0023E1F0705
:101F5000B9F781E06C96E8E00C946C25CF93C82F1C
:101F6000682F86E094E00E941C1C909192039C27AD
:101F700090939203CF910895A1E0B0E0E2ECFFE0EE
:101F80000C94562599830E94AE0F9981892F0E9447
:101F9000AE0F2196E2E00C9472251F93CF93DF934E
:101FA000182FEB011092920365EB86E094E00E94FB
:101FB0001C1C62E686E094E00E941C1C812F0E949B
:101FC000AE0FCE010E94BC0FDF91CF911F910895FB
:101FD0006091920386E094E00E941C1C0895A1E2A7
:101FE000B0E0E5EFFFE00C9452257B018A018C30D4
:101FF00009F453C108F040C0863009F4BCC018F59C
:10200000833009F491C070F4813009F472C08230D9
:1020100009F048C26BE170E082E00E94CD0F07EC4E
:1020200013E078C0843009F487C0853009F03AC2E3
:102030006091710370E0660F771F85E00E94CD0FFD
:1020400002E713E086C0893009F4A7C070F4873036
:1020500009F49BC0883009F025C261E070E088E097
:102060000E94CD0F8091FC0323C28A3009F4CAC0BC
:102070008B3009F4F2C016C28A3609F475C1D8F45F
:10208000873609F43AC138F4853609F40EC186362C
:1020900009F41FC107C2883609F437C1893609F02F
:1020A00001C261E070E089E60E94CD0F0E94EA0162
:1020B0000E942F02F5C18D3609F4D4C138F48B3655
:1020C00009F491C18C3609F49AC1ECC18E3609F439
:1020D000DCC1873C09F0E6C161E070E087EC0E945A
:1020E000CD0F81E00E94AE0F0E94E80F1092930383
:1020F000E3C169E270E081E00E94CD0F0EE913E0D8
:10210000F80181918F010E94AE0FF3E0073C1F0799
:10211000B9F7D0C1F80181918F010E94AE0FF3E0B1
:10212000023E1F07B9F7C6C161E070E083E00E947C
:10213000CD0F0E940B0FBCC161E070E084E00E94F3
:10214000CD0F81E00E94AE0F0E94E80F0E943E0D6D
:10215000B3C18091710390E0880F991F98012257B5
:1021600033402817390708F0A5C1F80181918F0184
:102170000E94AE0FEECF62E070E086E00E94CD0FCD
:1021800081E893E00E94BC0F95C161E070E087E0B8
:102190000E94CD0F809170038BC186E6898361E038
:1021A000CE0101960E9460070E94DE0683E08093C4
:1021B0009B0368EC70E080E090E00E94611A8091DF
:1021C0009B038430D9F48FE70E94FC040E940F0522
:1021D0008983863469F460E270E089E00E94CD0F63
:1021E00010E20E940F050E94AE0F1150D1F762C19C
:1021F00061E070E089E00E94CD0F52C161E070E0C3
:1022000089E053C169E170E08AE00E94CD0F82E06D
:102210008093E20320919A038091E7039091E80371
:10222000A091E903B091EA03222311F0806801C074
:102230008F778093E7039093E803A093E903B0932B
:10224000EA0302EE13E0F80181918F010E94AE0FC4
:10225000F3E00B3F1F07B9F72DC161E270E08BE09F
:102260000E94CD0F80913A038F3F39F080913A035D
:1022700091E0980F90933A0302C080913A030E9434
:10228000AE0F10E0812F0E94190D0E948D040E9454
:10229000BC0F1F5F1031B1F70DC161E070E08CE041
:1022A0000E94CD0F8091FB0303C161E070E085E6E1
:1022B0000E94CD0F89E2E816F10409F0F8C0D801B8
:1022C000EEE9F3E08D91819383E0E73CF807D1F7E5
:1022D000E7C061E070E086E60E94CD0FEBE1EE160C
:1022E000F10409F0E4C0D801E7ECF3E08D918193AB
:1022F00083E0E23EF807D1F7D3C061E070E087E603
:102300000E94CD0F0E94C408CBC061E070E088E657
:102310000E94CD0F85E789838BE1E7ECF3E0DE01D6
:10232000129601900D928A95E1F76CE1CE0101962B
:102330000E9460070E94DE0683E080939B0360E2B8
:1023400073E080E090E00E94611A80919B038430EA
:1023500009F0ADC08FE70E94FC040E940F0589833D
:10236000853509F0A4C09CC061E070E08AE60E9457
:10237000CD0F89E6898361E0CE0101960E94600756
:102380000E94DE0683E080939B0360E273E080E0BE
:1023900090E00E94611A80919B03843009F087C00D
:1023A0008FE70E94FC040E940F0589838E010E5F57
:1023B0001F4F7E01EDE1EE0EF11C0E940F05F801AA
:1023C00081938F01EE15FF05C1F78BE1FE01329677
:1023D000A7ECB3E001900D928A95E1F789818934E9
:1023E00009F065C05DC061E070E08BE60E94CD0F32
:1023F000F80180818093FC030E94CD0851C061E008
:1024000070E08CE60E94CD0FF0E2EF16F10461F46B
:1024100087E6898380E2F801DE01129601900D9231
:102420008A95E1F761E203C087E4898361E0CE0128
:1024300001960E9460070E94DE0683E080939B0362
:102440006CE474E080E090E00E94611A80919B034C
:10245000843069F58FE70E94FC040E940F058734E1
:1024600031F51EC061E070E08DE60E94CD0F89E17C
:10247000E816F104E1F4D801E2EEF3E08D918193E6
:1024800083E0EB3FF807D1F70BC061E070E08EE628
:102490000E94CD0FF80180818093FB030E94AE085B
:1024A00081E006C061E070E08AEC0E94CD0F80E020
:1024B0000E94AE0F0E94E80FA196E6E00C946E25F4
:1024C000A0E0B0E0E6E6F2E10C945025CAE5D2E0E7
:1024D00014E606E035E0F32E44E0E42E53E0D52E7A
:1024E00062E0C62E86E094E00E94AB1B892B09F4C3
:1024F0009BC086E094E00E94CF1B282F8093C502EA
:102500004091C40250E04730510560F7FA01EA5AA1
:10251000FF4F0C947D25853B29F781E08093C40211
:10252000E1CF823609F07DC0C092C402DBCF809338
:10253000C3028093C202D092C402D4CF9C0133273D
:102540003093C1022093C0029091C20298279093C9
:10255000C202E092C402C6CF382F22274091C002A7
:102560005091C102242B352B3093C1022093C0021D
:102570009091C20298279093C202F092C40225362D
:10258000310508F4AFCF61E070E08CEC0E94CD0F14
:1025900081E00E94AE0F0E94E80F43C02091BE026E
:1025A0003091BF02F901E65AFD4F80839091C2023B
:1025B00098279093C202C90101969093BF0280931D
:1025C000BE022091C0023091C1028217930708F425
:1025D00089CF0093C40286CF8091C20282130BC0C0
:1025E0006091BE027091BF024AE552E08091C30241
:1025F0000E94EF0F0DC062E070E08BEC0E94CD0FE7
:102600008091C3020E94AE0F809192030E94AE0F90
:10261000FE01812F11928A95E9F71092BF02109264
:10262000BE021092C4025ECFCDB7DEB7E8E00C94D4
:102630006C2581E08093930380919303882349F074
:1026400086E094E00E94AB1B892BB1F30E946012DC
:10265000F3CF0895AAE2B0E0E0E3F3E10C944E2555
:102660000E94321A6B017C0181E00E94030686E021
:1026700094E00E94AB1B892B29F086E094E00E9435
:10268000CF1BF5CF5F9811E072E6B72EE9E2AE2ED0
:1026900003E00E94321A6C197D098E099F09693C7A
:1026A000710581059105D0F11123C1F10E94321A03
:1026B0006B017C01469A80ED97E00E94FF02B9828F
:1026C000EEE9F3E0DE0112968A2D01900D928A95D3
:1026D000E1F76AE2CE0101960E946007469880E029
:1026E00090E00E94FF0200939B030E94DE0662E3DB
:1026F00070E080E090E00E94611A80919B0384303A
:1027000061F400939B038FE70E94FC040E940F0575
:1027100011E0823419F410E001C011E082E10E945E
:10272000821B892B81F411E00EC05F9A469A86E0E5
:1027300094E00E94CF1B8D309105A9F05CF40A97BC
:1027400091F05F98469886E094E00E94AB1B892B3D
:1027500061F79FCF8332910569F08234910589F743
:102760000E941913EECF66ED70E086E094E00E94BF
:10277000341DE7CF0E943E0DE4CF8F929F92AF921F
:10278000BF92CF92DF92EF92FF921F93CF93DF938E
:1027900082E10E94821B892B09F089C068EC70E0FD
:1027A00080E090E00E94611A80E090E00E94FF02C9
:1027B0000E94321A4B015C016B017C0180ECC80E57
:1027C00082E1D81EE11CF11C0E94321A6C157D05B5
:1027D0008E059F0530F482E10E94821B892BA1F3B4
:1027E00064C082E10E94821B892B09F05EC080EDEB
:1027F00097E00E94FF020E94321A6B017C01D0E038
:10280000C1E088E4880E86E2981EA11CB11C11E08C
:1028100082E10E94821B892B21F58C149D04AE0459
:10282000BF0430F480ED97E00E94FF02D1E0F0CFCA
:102830000E94321A6C197D098E099F09693C710545
:102840008105910528F30E94321A6B017C01C12792
:1028500019F080ED97E002C080E090E00E94FF0256
:10286000D7CF80E090E00E94FF02DD23B9F0809195
:10287000FB0390E0019665E070E00E94F1248093F4
:10288000FB030E94AE080E940E0B0E94CD0864EF6D
:1028900071E080E090E00E94611A09C080E00E942F
:1028A0004F020E942B090E94C4080E942A13DF9144
:1028B000CF911F91FF90EF90DF90CF90BF90AF909E
:1028C0009F908F900895CF92DF92EF92FF9280E0D9
:1028D0000E945C030E94200361E086E00E94161BB8
:1028E00061E085E00E94161B60E082E10E94161BF9
:1028F00060E084E00E94161B61E084E00E944F1BB0
:102900000E94F30260E070E086E094E00E94A11C67
:102910000E940E0B0E94CD080E94F30A8FEF809355
:102920003A030E942C0378940E94321A6B017C01B6
:1029300080913A038F3F59F40E94321A6C197D0935
:102940008E099F09603D77408105910588F380EDF0
:1029500097E00E94FF0261E082E10E944F1B5F9AB4
:1029600086E094E00E94AB1B892B29F086E094E07E
:102970000E94CF1BF5CF6EEE71E086E094E00E94DE
:10298000151D81E893E00E94B50765E072E086E0DE
:1029900094E00E94151D4AE050E066E070E086E099
:1029A00094E00E94DC1D62E370E080E090E00E9411
:1029B000611A86E094E00E94AB1B04970CF186E05C
:1029C00094E00E94CF1B82349105D1F486E094E01C
:1029D0000E94CF1B8E34910599F486E094E00E940A
:1029E000CF1B8434910561F486E094E00E94CF1BF4
:1029F000819731F480E090E00E94FF020E942A1348
:102A000040919F035091A0036091A1037091A20394
:102A1000DB01CA010197A109B1090497A105B1051C
:102A200068F440933903433029F440EA56E861E002
:102A300070E004C040E052EC61E070E088E594E0B2
:102A40000E94711F0E94BD135F9880E090E00E9479
:102A5000FF020E94F30A109255038091E70383FF5F
:102A600011C08091B303882351F08091BA03882369
:102A700031F08091C103882311F087E001C085E027
:102A80008093550380E00E940306809156030E94C4
:102A900037050E94DE061092CF021092CE021092ED
:102AA000CD02F12C8091FC038F15B0F062E370E051
:102AB00080E090E00E94611A80ED97E00E94FF02A2
:102AC00062E370E080E090E00E94611A80E090E0B4
:102AD0000E94FF02F394E6CF8091C60384FF08C0F2
:102AE000982F987181E0983109F080E00E94E70802
:102AF0008FE00E945C03FF90EF90DF90CF900895ED
:102B0000EF92FF920F931F93CF93DF938C016EE7A9
:102B100070E088E594E00E94C901E801F12CF0E240
:102B2000EF2E8E0188818D57823048F46DE770E07A
:102B300088E594E00E94C90188818E2588832196CA
:102B4000F801608188E594E00E94831EF394F9E027
:102B5000FF12E7CF6EE770E088E594E00E94C901BC
:102B6000CDB7DEB7E6E00C946E25A9E0B0E0EBEB64
:102B7000F5E10C9456259091570391110EC09EEFEC
:102B800099838A836B8350E0559547954C832D83B9
:102B9000198618861F821E822EC040915C03842FE6
:102BA00090E0B4E095958795BA95E1F7242F2F70C2
:102BB00030E08217930719F18DEF89831B82FE01A4
:102BC000349650E0842F90E0A4E095958795AA95DF
:102BD000E1F7242F2F7030E08217930749F0DC01D2
:102BE000A35ABC4F8C918193405F5F5F563051F781
:102BF00040935C035A83CE0101960E948015809118
:102C0000570390E0019666E070E00E94F124809303
:102C100057032996E2E00C947225A0E0B0E0E3E1CE
:102C2000F6E10C944F256C016EE770E088E594E0C6
:102C30000E94C9018601E12CF12CC0E0D0E030E215
:102C4000B32EF801608183E8860F823078F46DE757
:102C500070E088E594E00E94C901F80160816B256D
:102C600070E088E594E00E94C90104C088E594E022
:102C70000E94831EE114F10459F0F80180819E0145
:102C8000280F311DC901C92FDD27C80FD91FDD2726
:102C90003FEFE31AF30A89E0E816F10459F028E05F
:102CA000E216F10421F48C2F8095F60180870F5FE6
:102CB0001F4FC7CFCDB7DEB7E9E00C946B25A9E075
:102CC000B0E0E5E6F6E10C945625E82F362F80912A
:102CD000570390E0019664E270E00E94F124809333
:102CE000570358E9598350E15A83813089F048F0FD
:102CF0008230B9F08330D9F48B8381EF8C833D83AC
:102D000019C085E08B8381EF8C832F5F2D8312C0E8
:102D10008B8381EF8C8384E6489FA00111245D831F
:102D200009C084E08B8381EF8C83ED8303C00E9414
:102D3000240904C0CE0101960E940D162996E2E0F6
:102D40000C947225A2E0B0E0E8EAF6E10C944B2581
:102D5000182F762E2A8349830E943E1A6B017C012C
:102D600080916D038090580390905903A0905A036E
:102D7000B0905B032A8149818823C1F0D701C60145
:102D800088199909AA09BB094C015D0191EE8916C0
:102D90009EE29906A104B10420F1241708F4422F01
:102DA000202F672D812F0E945F1613C0D701C60107
:102DB00088199909AA09BB094C015D0191E389169B
:102DC00095E79906A104B10460F0672D812F0E9458
:102DD000B515C0925803D0925903E0925A03F0926D
:102DE0005B032296EDE00C946725A2E2B0E0EBEFE6
:102DF000F6E10C944C258CE00E941E0581110DC05B
:102E00006DE072E086E094E00E94461D5F9A80E0EB
:102E10000E9403060E94DE065F9888E594E00E9407
:102E2000291E892B01F188E594E00E94561E90919D
:102E30003903992319F00E94210BEFCF4091CE0264
:102E400050E09A012F5F3F4F2F7133276091CF02DF
:102E500070E02617370709F3FA01E752FD4F808328
:102E60002093CE02DACF80913903811106C0809180
:102E70009B03843009F094C00DC086E094E00E946A
:102E8000AB1B892BA1F386E094E00E94CF1B0E942C
:102E9000210BF3CF0E943E1A611571058105910542
:102EA00049F06093470370934803809349039093DC
:102EB0004A030CC081E090E0A0E0B0E080934703BB
:102EC00090934803A0934903B0934A0380913D0334
:102ED00090913E03816090933E0380933D0383E095
:102EE00080939B038FE70E94FC0409EF12E00E948D
:102EF0000F05F80181938F01F3E002301F07B9F746
:102F0000209102038091F902982F922796FF3BC0EF
:102F100090E4922790930203982F98739833F1F4DA
:102F200010E0212F30E08091F902877090E0821745
:102F300093074CF11F5F2091C603812F90E0FC01A5
:102F4000E750FD4F24FF04C080810E940609E9CFAD
:102F5000608188E594E00E94831EE3CF8F7399F42B
:102F60008091FA02809346038091FB028093440390
:102F70008091FC02809343038091FF0290E0909344
:102F80003C0380933B038091CD02813019F482E0B1
:102F90008093CD028091CD02833011F41092CD0246
:102FA0000E943E1A6B017C0180913F039091400387
:102FB000A0914103B09142030097A105B105C9F06A
:102FC000A7019601281B390B4A0B5B0BDA01C901DB
:102FD000883B9B40A105B10560F00E944D058093A0
:102FE000450310923F031092400310924103109248
:102FF000420380914B0390914C03A0914D03B091FB
:103000004E0346015701881A990AAA0ABB0A8EE99B
:1030100093E00E94780386169706A806B90608F47E
:10302000A8C0C0924B03D0924C03E0924D03F092A3
:103030004E030E94C00180913A038830A0F0809135
:10304000E7039091E803A091E903B091EA036CE1F2
:10305000B695A795979587956A95D1F7892B8A2B71
:103060008B2B09F0A4C180913A038F5F80933A03C0
:103070008091470390914803A0914903B0914A037E
:103080000097A105B105F1F0C81AD90AEA0AFB0AAE
:103090008EE993E00E9478036C157D058E059F05EF
:1030A00008F006C18091E70384FD04C080ED97E03D
:1030B0000E94FF02109247031092480310924903A6
:1030C00010924A0390910203907C909302035091D6
:1030D000CE028091CF022091CD02581709F405C18C
:1030E000223009F002C1905890930203E091C60388
:1030F000E770F0E0E45EFD4F6081693008F0DDC00C
:10310000615040E04613DBC08093CF0287E3840F19
:1031100090910203892B809302034093D00283E0B5
:103120008093CD02469A8091AB0390915503911103
:103130002FC10E94FE05809156030E943705E09141
:10314000C603E770F0E0E45EFD4F608182E093E04B
:103150000E941907E0915603EF5FE0935603E831B0
:1031600009F422C1F0E0E256FC4F8785882309F478
:103170001BC10E948807813069F58091C603887160
:1031800049F180913D0390913E03880F991F9093E0
:103190003E0380933D0383E080939B030E94DE0601
:1031A0000E943E1A60933F03709340038093410353
:1031B00090934203672B682B692B61F481E090E0C8
:1031C000A0E0B0E080933F0390934003A0934103BD
:1031D000B09342038091C60384FF1FC080913D03DA
:1031E00090913E038E7F0E94AE04182F60913B03A6
:1031F000809146030E94170B482F612F8091450351
:1032000049A30E94170B0091FC03282F49A160914C
:103210004303809144030E94A21646988091530371
:103220008130C1F018F08230B1F1CEC082E10E944D
:10323000821B892B09F0C8C081E0809353030E9450
:10324000321A60934F03709350038093510390930D
:103250005203BAC082E10E94821B892B31F50E9481
:10326000321AC0904F03D0905003E0905103F09079
:1032700052036C197D098E099F09693E73408105CF
:10328000910508F4A1C082E08093530380ED97E09C
:103290000E94FF0299C082E10E94821B892B09F4DF
:1032A00093C080E090E00E94FF02109253038CC014
:1032B00080E090E00E94FF0205CF68E022CF8517F2
:1032C00009F422CF4F5F242F30E090E0F901EE5F48
:1032D000FC4FDC01A752BD4F7C917083F901E05394
:1032E000FD4F708301968F710DCF2430B1F4209182
:1032F000D00281ED92E0A3E0B3E0FC013E2F381B49
:10330000321718F431913D93F9CF87E3820F9091F2
:103310000203892B8093020302CF809153038230F2
:1033200069F49160909302035F9A5BEEE52E53E09F
:10333000F52E8E010F5F1F4FB80110C05F9880916E
:10334000CD02811103C081E08093CD028091CD0236
:10335000833059F784E08093CD02E7CFF701819164
:103360007F0169A37AA30E94190DF80181939193BB
:103370008F0169A17AA1FBEFEF16F3E0FF0671F769
:103380008091C60343E053E087700E94FD03CACEDC
:10339000882309F4CECE2091540331E0320F3093CC
:1033A00054032913C6CE0CC010925603E2CE80916E
:1033B0003A03883009F45F9A89E080933A03D9CEC2
:1033C000109254038150B5CEA296ECE00C9468257F
:1033D0001F920F920FB60F9211242F933F938F934A
:1033E0009F93AF93BF938091FE039091FF03A091B1
:1033F0000004B09101043091FD0323E0230F2D3729
:1034000020F40196A11DB11D05C026E8230F0296E8
:10341000A11DB11D2093FD038093FE039093FF0334
:10342000A0930004B09301048091020490910304DE
:10343000A0910404B09105040196A11DB11D8093D3
:10344000020490930304A0930404B0930504BF9175
:10345000AF919F918F913F912F910F900FBE0F9041
:103460001F9018952FB7F8946091FE037091FF0399
:1034700080910004909101042FBF08953FB7F89404
:103480008091020490910304A0910404B09105047A
:1034900026B5A89B05C02F3F19F00196A11DB11DAF
:1034A0003FBF6627782F892F9A2F620F711D811DCC
:1034B000911D42E0660F771F881F991F4A95D1F72B
:1034C0000895CF92DF92EF92FF92CF93DF936B013B
:1034D0007C010E943E1AEB01C114D104E104F10405
:1034E00079F00E943E1A6C1B7D0B683E7340A0F37E
:1034F00081E0C81AD108E108F108C851DC4FECCFCF
:10350000DF91CF91FF90EF90DF90CF900895789466
:1035100084B5826084BD84B5816084BD85B58260D8
:1035200085BD85B5816085BDEEE6F0E08081816076
:103530008083E1E8F0E01082808182608083808176
:1035400081608083E0E8F0E0808181608083E1E950
:10355000F0E0808182608083808181608083E0E907
:10356000F0E0808181608083E1ECF0E08081846024
:103570008083808182608083808181608083E3ECAE
:10358000F0E0808181608083E0ECF0E08081826007
:103590008083E2ECF0E0808181608083EAE7F0E004
:1035A000808184608083808182608083808181606B
:1035B0008083808180688083089590E0FC0131974A
:1035C000EE30F10590F5E35AFF4F0C947D25809184
:1035D00080008F7703C0809180008F7D8093800072
:1035E000089584B58F7702C084B58F7D84BD08951A
:1035F000809190008F7707C0809190008F7D03C0ED
:1036000080919000877F8093900008958091C00002
:103610008F7703C08091C0008F7D8093C000089594
:103620008091C200877F8093C2000895CF93DF937B
:1036300090E0FC01E75EFE4F2491FC01E95CFE4F47
:103640008491882349F190E0880F991FFC01EF587D
:10365000FE4FA591B4918D599E4FFC01C591D49117
:103660009FB7611108C0F8948C91209582238C93A8
:10367000888182230AC0623051F4F8948C91322FF1
:10368000309583238C938881822B888304C0F8949F
:103690008C91822B8C939FBFDF91CF910895A1E0F5
:1036A000B0E0E5E5FBE10C945425282F30E0F9016A
:1036B000E550FF4F8491F901E75EFE4F1491F90147
:1036C000E95CFE4F04910023C9F0882321F069834F
:1036D0000E94DD1A6981E02FF0E0EE0FFF1FED5927
:1036E000FE4FA591B4919FB7F8948C91611103C0DE
:1036F0001095812301C0812B8C939FBF2196E4E01C
:103700000C947025CF93DF93282F30E0F901E5501A
:10371000FF4F8491F901E75EFE4FD491F901E95C16
:10372000FE4FC491CC2391F081110E94DD1AEC2F41
:10373000F0E0EE0FFF1FEB5AFE4FA591B4912C91D4
:103740002D2381E090E021F480E002C080E090E051
:10375000DF91CF9108958091540490915504209168
:10376000560430915704821B930B8F739927089549
:10377000209154043091550480915604909157043F
:103780002817390749F0E0915604F0915704EC5E90
:10379000FB4F808190E008958FEF9FEF0895209177
:1037A0005404309155048091560490915704281781
:1037B0003907A9F0E0915604F0915704EC5EFB4FF5
:1037C000808120915604309157042F5F3F4F2F7313
:1037D0003327309357042093560490E008958FEFD9
:1037E0009FEF0895CF93DF93C0915404D091550477
:1037F0002196CF73DD278091560490915704C81706
:10380000D90799F082E00E94A7208F3F2FEF9207FF
:1038100061F0E0915404F0915504EC5EFB4F80831D
:10382000D0935504C0935404DFCFDF91CF91089516
:1038300083E00E94F2220895A1E0B0E0E2E2FCE120
:103840000C9454258C0169838091A401882359F03C
:1038500041E050E0BE016F5F7F4F83E00E94DA20BD
:10386000181619063CF081E090E0F80193838283FA
:1038700080E090E02196E4E00C947025FC0120812A
:103880002E5F208342E450E06FE771E080E80E9401
:103890005A210895FC0181819081913A59F4813235
:1038A00009F04BC047E050E06DE971E080E00E9414
:1038B0005A2145C0913209F040C0803239F467E0A6
:1038C00070E08DE991E00E949E2139C0823209F0BA
:1038D00034C082818093A40180919D0190919E01CA
:1038E000A0919F01B091A001803B9440A105B1053A
:1038F00031F58091A40180FD12C087E797E790938E
:103900000108809300082BE088E190E00FB6F8945E
:10391000A895809360000FBE2093600010C088E1DE
:103920000FB6F89480936000109260000FBEA895C7
:10393000109201081092000802C080E0089581E012
:1039400008950895109209041092080488EE93E0F7
:10395000A0E0B0E080930A0490930B04A0930C04C1
:10396000B0930D048EE292E09093070480930604D6
:103970000895A0E0B0E0EFEBFCE10C9450256C0161
:103980007A01EB01E60EF71E00E010E0CE15DF0530
:1039900061F06991D601ED91FC910190F081E02DEB
:1039A000C6010995080F191FF1CFC801CDB7DEB7C1
:1039B000E8E00C946C256115710589F0DB010D9030
:1039C0000020E9F7AD0141505109461B570BDC01BE
:1039D000ED91FC910280F381E02D0995089580E03E
:1039E00090E00895EF92FF920F931F93CF93DF9390
:1039F0008C01FB01C0E0D0E064917F018FEFE81AF9
:103A0000F80A662361F0D801ED91FC910190F081F4
:103A1000E02DC8010995C80FD91FF701EDCFCE01E0
:103A2000CDB7DEB7E6E00C946E250E94DB1C08954E
:103A3000DC01ED91FC910190F081E02D0995089554
:103A40000F931F93CF93DF93EC016DE00E94181D3D
:103A50008C016AE0CE010E94181D800F911FDF913A
:103A6000CF911F910F9108950F931F93CF93DF93E1
:103A7000EC010E94F21C8C01CE010E94201D800FDF
:103A8000911FDF91CF911F910F9108950F931F9375
:103A9000CF93DF93EC010E94DB1C8C01CE010E94CE
:103AA000201D800F911FDF91CF911F910F910895DD
:103AB0000F931F93CF93DF93EC010E94181D8C018D
:103AC000CE010E94201D800F911FDF91CF911F9189
:103AD0000F910895A1E2B0E0E0E7FDE10C944C25E0
:103AE0007C01C42EE52FCB01D22E19A221E02D1589
:103AF00010F02AE0D22E8E010F5D1F4F8D2C912CDD
:103B0000A12CB12C6C2D7E2FA50194010E940525BE
:103B10008C2DD29E80191124015011098A3010F485
:103B2000805D01C0895CF801808321153105410564
:103B3000510521F0C22EE32FCA01E4CFB801C7011D
:103B40000E94DB1CA196ECE00C946825A0E0B0E09C
:103B5000ECEAFDE10C945025EC016A017B01211592
:103B6000310541F4E881F9810190F081E02D642F65
:103B700009951DC02A303105A9F477FF12C06DE206
:103B80000E94181D8C0144275527BA014C195D0964
:103B90006E097F092AE0CE010E946A1D800F911FE5
:103BA00006C02AE0B701A601CE010E946A1DCDB76A
:103BB000DEB7E8E00C946C250F931F93CF93DF934F
:103BC000EC019A01AB01662757FD6095762F0E94A4
:103BD000A61D8C01CE010E94201D800F911FDF9138
:103BE000CF911F910F9108952115310549F4DC0102
:103BF000ED91FC910190F081E02D642F09950895DD
:103C00000E946A1D08959A01462F50E060E070E01E
:103C10000E94F41D08959A01AB0160E070E00E94DB
:103C2000F41D08950F931F93CF93DF93EC019A0136
:103C3000462F50E060E070E00E94F41D8C01CE0140
:103C40000E94201D800F911FDF91CF911F910F9136
:103C50000895FC0124853585F901E05CFF4F8081E2
:103C60009181F901EE5BFF4F20813181821B930B23
:103C70008F7399270895FC0184859585FC01E05C8C
:103C8000FF4F40815181FC01EE5BFF4F208131816C
:103C90004217530741F00190F081E02DE80FF91F22
:103CA000808190E008958FEF9FEF0895FC01848557
:103CB0009585FC01E05CFF4F40815181FC01EE5B8A
:103CC000FF4F208131814217530779F0A081B181E4
:103CD000A80FB91F8C91208131812F5F3F4F2F7327
:103CE00033273183208390E008958FEF9FEF08956D
:103CF000FC0181A1882329F0A489B5898C9186FFD4
:103D0000FBCF11A20895CF93DF93FC012685378561
:103D1000D901A05CBF4F8D919C91119701968F7333
:103D20009927E901CE5BDF4F4881598184179507B8
:103D3000D9F30D90BC91A02DA20FB31F6C93A68553
:103D4000B785A05CBF4F11969C938E93A689B789C7
:103D50002C9181E090E0078C02C0880F991F0A9493
:103D6000E2F7282B2C9381E081A30488F589E02DCC
:103D700080818064808381E090E0DF91CF9108951D
:103D800008951F920F920FB60F9211242F933F9315
:103D90004F938F939F93EF93FF938091C80082FD81
:103DA0001CC04091CE008091FE049091FF040196CA
:103DB0008F73992720910005309101058217930791
:103DC00071F0E091FE04F091FF04E254FB4F408358
:103DD0009093FF048093FE0402C08091CE00FF9177
:103DE000EF919F918F914F913F912F910F900FBE27
:103DF0000F901F90189588E594E00E94291E892B4A
:103E000011F00E94C01E08951F920F920FB60F92DC
:103E100011242F933F938F939F93EF93FF932091C0
:103E2000BA043091BB048091BC049091BD04281762
:103E3000390731F48091C9008F7D8093C90014C087
:103E4000E091BC04F091BD04E658FB4F20818091C5
:103E5000BC049091BD0401968F7399279093BD0483
:103E60008093BC042093CE00FF91EF919F918F919E
:103E70003F912F910F900FBE0F901F901895A0E0CB
:103E8000B0E0E5E4FFE10C944C25FC0113821282C2
:103E900088EE93E0A0E0B0E084839583A683B783A7
:103EA00080E492E091838083758764875787468793
:103EB000318B208B138B028BF58AE48AD78AC68AD2
:103EC000B18EA08E938E828E8F85848F8889858F08
:103ED0008989868F8A89878F8B8980A3ECE00C94EF
:103EE0006825CF92DF92EF92FF92CF93DF93EC01A0
:103EF0006A017B01411581EE580761057105F9F0F2
:103F0000EC89FD8981E090E008A002C0880F991F2C
:103F10000A94E2F7808360E079E08DE390E0A70106
:103F200096010E94052521503109410951095695F4
:103F3000479537952795211580E1380798F0EC894A
:103F4000FD89108260E874E88EE190E0A701960197
:103F50000E9405252150310941095109569547957F
:103F600037952795E889F9893083EA89FB89208389
:103F700019A2EE89FF89408181E090E09C010C8CC0
:103F800002C0220F331F0A94E2F7422B4083EE89CE
:103F9000FF8940819C010D8C02C0220F331F0A94BF
:103FA000E2F7422B4083EE89FF8940819C010E8C11
:103FB00002C0220F331F0A94E2F7422B4083EE899E
:103FC000FF8920810F8C02C0880F991F0A94E2F7A5
:103FD000809582238083DF91CF91FF90EF90DF90D7
:103FE000CF9008958F929F92AF92BF92CF92DF921F
:103FF000EF92FF920F931F9381E08F9385E08F9351
:1040000087E08F9383E08F9384E08F93EEEC8E2E86
:10401000912CFAECAF2EB12CA9ECCA2ED12CB8EC15
:10402000EB2EF12C0CEC10E02DEC30E04AE754E0E4
:104030006EEB74E088E594E00E943F1F0F900F90B4
:104040000F900F900F901F910F91FF90EF90DF90C6
:10405000CF90BF90AF909F908F9008950E94871A45
:1040600082E095E00E94FC220E946314CBEFDEE127
:104070000E94F5162097E1F30E94FB1EF9CF6150D4
:1040800030F02091F100FC0120830196F8CF2898B0
:1040900084E68093090508952FB7FC012083F894E6
:1040A00067706093E9000895A1E0B0E0EAE5F0E20E
:1040B0000C945625682FCE0101960E944C208091C9
:1040C000F20099819FBF2196E2E00C947225A2E054
:1040D000B0E0EDE6F0E20C945325F62E8A019091C3
:1040E0000805992311F057FF03C08FEF9FEF2BC0F6
:1040F000682FCE0101967A830E944C208091F200B5
:1041000090E0A8017A81801791070CF4AC01EF2DA3
:10411000F72FF40E84E6FE1639F0289880930905EF
:104120009091F1009193F7CF4115510521F08091C5
:10413000F200882321F089818FBFCA0104C08BE679
:104140008093E800F8CF2296E5E00C946F25A1E07B
:10415000B0E0EDEAF0E20C94562541E050E0BE01FB
:104160006F5F7F4F0E946720019719F4898190E06B
:1041700002C08FEF9FEF2196E2E00C947225A1E040
:10418000B0E0E5ECF0E20C945625682FCE010196E4
:104190000E944C209091E800892F807295FF04C006
:1041A0009091F20080E4891B99819FBF2196E2E003
:1041B0000C947225A1E0B0E0E0EEF0E20C9448250A
:1041C000582E7B01A42E952E80910805882369F036
:1041D000042F152F8AEFB82E852D8072782E9AE342
:1041E000892E852D8074682E11C08FEF9FEF53C0EC
:1041F000852D0E94BF20482E81110CC0BA94A9F3CE
:1042000061E070E080E090E00E94611A0115110504
:1042100079F737C0282F30E0021713070CF4402E2F
:10422000C42CD12C0C191D09652DCE0101960E94BC
:104230004C20772039F04A948FEF4816B1F0109255
:10424000F100F9CFF701842D57FE07C0815058F0D7
:1042500094919093F1003196F9CF815020F0919193
:104260009093F100FACFEC0CFD1C8091E80085FFE3
:104270000FC00115110511F461100AC089818FBFAB
:10428000C5CF5D9884E680930A058A2D992D03C0D9
:104290008092E800F3CF2196E0E10C94642510921F
:1042A000E90010920705109206059093050580938A
:1042B00004050895CF93DF93FB0120E030E0DEEFAB
:1042C00024173507A1F187FF02C0C49101C0C08146
:1042D000A0910605B0910705609104057091050550
:1042E000A617B707B4F49091E8009570E1F39091A8
:1042F000E80092FD1EC0C093F10060910605709128
:1043000007056F5F7F4F6F737727672B11F4D0938B
:10431000E80060910605709107056F5F7F4F70930D
:104320000705609306052F5F3F4F3196C9CFC9013E
:1043300002C08FEF9FEFDF91CF910895A1E0B0E031
:10434000E4EAF1E20C945525162F2091E80022FFB3
:10435000FCCF612F79830E943F208BEF8093E80090
:10436000812F7981972F2196E3E00C947125A1E0AC
:10437000B0E0EDEBF1E20C9456251982CE010196E6
:104380000E943E1CCE0101960E949623898190E0F6
:104390002196E2E00C9472251F920F920FB60F92B5
:1043A0001124EF92FF920F931F932F933F934F93FC
:1043B0005F936F937F938F939F93AF93BF93EF938D
:1043C000FF93CF93DF93CDB7DEB76297DEBFCDBF4C
:1043D0001092E9008091E80083FFE7C068E0CE0119
:1043E0000A960E943F2082EF8093E8009A8597FF0B
:1043F00005C08091E80080FFFCCF03C08EEF809362
:10440000E800892F807609F0B5C08B85811105C041
:104410001092F1001092F100C1C0282F2D7F2130A1
:1044200009F4BCC0853049F48091E80080FFFCCFDE
:104430008C8580688093E300B1C0863009F072C03B
:104440002D85E888F988223071F580E090E02A8B8C
:104450000E944F210E94B72199E08E010F5F1F4FEC
:10446000F801392F11923A95E9F799832A892A831D
:1044700091E09E8390E898879AEF998720910605AE
:1044800030910705275F3F4F3C832B838D83C70106
:104490000E944F2149E050E0B80180E00E945A217B
:1044A0000E94B7217BC0C7012A8B0E944F212A8915
:1044B000223241F482E290E00E94A223892B09F08B
:1044C0006DC070C0213069F488899989089711F40A
:1044D0002093030580910305882389F066EC71E041
:1044E00016C0233009F05EC08C85882359F08230D5
:1044F00061F0813009F056C06AEE71E008C068EDE5
:1045000071E005C064E272E002C062E072E0611531
:10451000710509F447C0FB01449150E080E80E9416
:104520005A213CC0873009F43DC0883021F481E035
:104530008093F10033C0893089F5937099F5E2ECEE
:10454000F1E081E021E096E38093E9002093EB0025
:1045500034913093EC009093ED008F5F319685306D
:1045600099F78EE78093EA001092EA008C85809399
:10457000080514C0888999890E944F218E85811170
:1045800005C0CE010A960E944A1C06C0823051F432
:10459000CE010A960E94C423882321F08EEF8093D7
:1045A000E80003C081E28093EB0062960FB6F894B6
:1045B000DEBF0FBECDBFDF91CF91FF91EF91BF91D5
:1045C000AF919F918F917F916F915F914F913F91AB
:1045D0002F911F910F91FF90EF900F900FBE0F90B2
:1045E0001F9018958093E9008091F200882319F0BC
:1045F0008AE38093E80008951092080581E0809393
:10460000D70080EA8093D80082E189BD09B400FE1A
:10461000FDCF61E070E080E090E00E94611A80E9E7
:104620008093D8008CE08093E2001092E000559ACD
:10463000209A08951F920F920FB60F9211242F9374
:104640003F934F935F936F937F938F939F93AF931A
:10465000BF93EF93FF938091E1001092E10083FFFD
:104660000FC01092E90091E09093EB001092EC00E3
:1046700092E39093ED001092080598E09093F0007B
:1046800082FF26C083E00E94F22282E00E94542032
:10469000882321F086E094E00E94F21B80910A05B5
:1046A000882339F080910A05815080930A05882378
:1046B00069F080910905882359F08091090581509E
:1046C00080930905811104C0289A02C05D9AF1CF38
:1046D000FF91EF91BF91AF919F918F917F916F91DA
:1046E0005F914F913F912F910F900FBE0F901F90B0
:1046F0001895FF920F931F93CF93DF93EC01F62E43
:10470000E881F9810480F581E02D09958C01E8812B
:10471000F9810680F781E02D6F2DCE010995C80142
:104720009927CDB7DEB7E5E00C946F25FC01208119
:104730002F5F208349E150E068EA72E080E80E9440
:104740005A21089545E650E061EC72E080E80E944D
:104750005A210895A1E0B0E0E0EBF3E20C94522579
:1047600089838B017A0141E050E0BE016F5F7F4F8A
:1047700084E00E94DA20A701B80184E40E94DA20D4
:104780002196E6E00C946E25FC0191818081813AAE
:1047900031F481E0913091F0933089F411C081328D
:1047A00071F49B3021F482818093A60105C09A3078
:1047B00031F482818093A50181E00895089580E01D
:1047C0000895FC0110820895FC011382128220E5F5
:1047D00032E031832083089548E050E082E00E9477
:1047E000AA230895CF93DF93DC01683818F0E8E737
:1047F000E60F25C0E62FF0E067FF11C0E058F10991
:1048000081E090E001C0880FEA95EAF714969C9148
:104810001497982B14969C931497E0E010C0E85DD1
:10482000FD4FE491EE2309F440C0E7FF08C0149661
:104830008C911497826014968C931497EF77169648
:104840008C9116978E1741F117968C9117978E17AA
:1048500019F118968C9118978E17F1F019968C9182
:1048600019978E17C9F01A968C911A978E17A1F086
:104870001B968C911B978E1779F080E090E0ED01EC
:10488000C80FD91F2E81211102C0EE8305C00196E9
:1048900086309105A1F709C0BD016C5F7F4FCD0146
:1048A0000E94EC2381E090E008C081E090E0139644
:1048B0009C938E93129780E090E0DF91CF910895C2
:1048C000683818F0E8E7E60F25C0E62FF0E067FF4C
:1048D00012C0E058F10921E030E001C0220FEA9552
:1048E000EAF72095DC0114963C9114973223149634
:1048F0003C93E0E00FC0E85DFD4FE491EE2329F129
:10490000E7FF08C0DC0114962C9114972D7F1496B4
:104910002C93EF7720E030E0EE2351F0DC01A20F82
:10492000B31F16964C9116974E1302C016961C9202
:104930002F5F3F4F2630310579F7BC016C5F7F4F09
:104940000E94EC2381E090E0089580E090E00895DB
:10495000FC01168217821086118612861386148235
:10496000BC016C5F7F4F0E94EC23089587E195E0C6
:104970000E94E1238BE095E00E94E4230895A29F2A
:10498000B001B39FC001A39F700D811D1124911D23
:10499000B29F700D811D1124911D08950E94BF24A6
:1049A000A59F900DB49F900DA49F800D911D112483
:1049B0000895B7FF0C94CE240E94CE24821B930B43
:1049C0000895DB018F939F930E94CE24BF91AF91F6
:1049D000A29F800D911DA39F900DB29F900D112459
:1049E000089597FB072E16F4009407D077FD09D0A1
:1049F0000E94832507FC05D03EF4909581959F4F3A
:104A00000895709561957F4F0895A1E21A2EAA1B13
:104A1000BB1BFD010DC0AA1FBB1FEE1FFF1FA2176E
:104A2000B307E407F50720F0A21BB30BE40BF50B6B
:104A3000661F771F881F991F1A9469F760957095F4
:104A4000809590959B01AC01BD01CF010895052E85
:104A500097FB1EF400940E943E2557FD07D00E944C
:104A6000052507FC03D04EF40C943E255095409547
:104A7000309521953F4F4F4F5F4F0895909580950A
:104A8000709561957F4F8F4F9F4F08952F923F9262
:104A90004F925F926F927F928F929F92AF92BF924E
:104AA000CF92DF92EF92FF920F931F93CF93DF93FA
:104AB000CDB7DEB7CA1BDB0B0FB6F894DEBF0FBE57
:104AC000CDBF09942A88398848885F846E847D84A4
:104AD0008C849B84AA84B984C884DF80EE80FD80A6
:104AE0000C811B81AA81B981CE0FD11D0FB6F8941C
:104AF000DEBF0FBECDBFED010895EE0FFF1F059085
:104B0000F491E02D0994AA1BBB1B51E107C0AA1F19
:104B1000BB1FA617B70710F0A61BB70B881F991F5E
:104B20005A95A9F780959095BC01CD0108958F9273
:104B30009F92AF92BF92CF92DF92EF92FF92CF936C
:104B4000DF93EC01688179818A819B816115710510
:104B50008105910521F464E279ED8BE597E02DE183
:104B600033EF41E050E00E94272549015A019B01A3
:104B7000AC01A7EAB1E40E94CE246B017C01ACEE4B
:104B8000B4EFA50194010E94DC24C60ED71EE81ED6
:104B9000F91EF7FE06C081E0C81AD108E10880E8D6
:104BA000F80AC882D982EA82FB82C701B6019F77E0
:104BB000DF91CF91FF90EF90DF90CF90BF90AF90BB
:104BC0009F908F9008950E949725089586E091E028
:104BD0000E949725089560930601709307018093C2
:104BE0000801909309010895F999FECF92BD81BD06
:104BF000F89A992780B50895262FF999FECF1FBA04
:104C000092BD81BD20BD0FB6F894FA9AF99A0FBEF5
:084C100001960895F894FFCF0E
:104C180000001805200001000000FF00020002004B
:104C2800020002000200020002000200020002006C
:104C380002000200020002000200028025000005B6
:104C4800400AA1204EA50020244EA52C2330C012D6
:104C580000001A400AA1204EA5001B1E27522C2333
:104C6800308025000005400AA1204EA50020244ED2
:104C7800A52C2330004B000006400AD0009D4900B7
:104C88007B289D492C233000E1000005400A45019E
:104C9800D7DC03B81E0EBF00232E48E801008A4067
:104CA8000A6001555502AD1E20000023C800E1002E
:104CB8000000000000010154582074696D656F758B
:104CC800742100456E746572696E67206164617055
:104CD80074697665206368616E6E656C2073656CB7
:104CE800656374696F6E2C207069636B696E673ACF
:104CF800007363616E6E6572206D6F6465004F703E
:104D0800656E4C52536E67205458207374617274E8
:104D1800696E672000206F6E20485720006D6F6411
:104D2800756C65206C6F636B65643F0000070B0C46
:104D380010111500160A13223129000000001C1C4E
:104D4800B91CAB1BCF1BB81B181CF21B00000000C2
:104D5800831EB91C291E561E3B1E781E000000002B
:0A4D68007923B91CF2236024A8246B
:00000001FF
